:100000008CC0B2C0AEC3B0C0AFC0AEC0ADC0ACC09B
:10001000ABC0AAC0A9C0A8C054C1A6C0A5C0814594
:1000200086468B479048944997609B619E62A16386
:10003000A464A765AA66AC67AE68B069B280B481F3
:10004000B682B883BA84BB84BD84FF21000000005F
:100050000000000000000000000023456C98C9FF6C
:10006000040714233764A0FFFFFFFFFFFFFFFFFF1C
:10007000FFFFFF00000000000000000023405F7A47
:10008000B4FFFFFFFFFFFF001400081400080E1468
:100090000004080E14000305080E140004080A0EDC
:1000A0001114000305080A0E1014000305080A0EB7
:1000B0001012140008000E00080E0004080E0003C1
:1000C00005080E0004080E1100080E1100F3F404D8
:1000D000080E10121400080A0C0E0F10121400085B
:1000E0000EED14000203040500041400040E1400B5
:1000F000040810140004080F1114000305080A0E68
:100100000004080A0E00EEEDECEB140E08040004E7
:10011000080E00EBECEDEEF3F41411241FBECFE556
:10012000D1E0DEBFCDBF20E0A0E6B0E001C01D926F
:10013000AB37B207E1F7ECE7F0E085E5808781E0D7
:10014000838314821282868311828BE0828788E502
:100150008387E1E6F0E08DEF87838EEF8583712C56
:1001600055245A94AFD018C34BCF1BBC19BC18BC34
:10017000089520ED37E0019720F0F9013197F1F76C
:10018000FACF089588EE93E0F4CF369A3699FECFF1
:1001900095B18091600089270895CF93C72D81E0A4
:1001A000870D8F73782E662D90E0E8D26FEF8C2F3D
:1001B00090E0CF91E3C2FF920F931F93CF93DF9311
:1001C000F82E0DE710E0CEE7D0E0F11005C0CE012B
:1001D000CDD2F801808304C0F8016081CE01CED277
:1001E00021970F5F1F4FC337D10579F7DF91CF916B
:1001F0001F910F91FF900895D0DF81E0DCCF811136
:1002000001C0B3CF815090E0FC01E45BFF4FE4916B
:10021000EBBDFC01E05AFF4FE491E9BDFC01EC5855
:10022000FF4F849188BD08950F931F93CF93C82FDC
:100230008B01CC2359F085E0E2DFC8019ADF95DF1E
:10024000C80197DFC80195DFC150F3CFCF911F914F
:100250000F910895EF92FF920F931F93CF93C8E0F1
:10026000E82EF12C062F10E084E1C9DFC70181DF01
:100270007CDFC8017EDFC150B9F7CF911F910F918C
:10028000FF90EF9008951F93CF93DF938FEA87B984
:1002900086EC86B91092600010E1C0E0D0E085E005
:1002A00090E067DF72DFC80FD11D1150C1F7CE019A
:1002B00024E0969587952A95E1F7DF91CF911F91DC
:1002C0000895189510927B0087E790E04FD285350E
:1002D00019F0612C91DF11C0712C872D90E046D26E
:1002E000682E8F3F19F080E066DF07C0872D91E010
:1002F000970D792E803488F3F6CF20918600C09137
:100300007F001091800080917D00882319F010E01B
:10031000C0E02AE12F5F90E040E050E0A8E8B0E0C4
:10032000222379F0BD016F5F7F4FFB013197E4918C
:10033000EE2319F0962F9A1BF6CF2150AD01DB0169
:10034000EFCF092F6C2F70E0A92FB0E0E02FF0E085
:10035000112321F09D012E1B3F0B05C09F01215051
:100360003109260F371F3197E40FF51FF4902559F7
:100370003F4FF901F082015049F79C0F909388009C
:10038000CC2371F0112329F0292F30E021503109BD
:1003900002C020E030E0F901E559FF4F41E0408321
:1003A00027E0290F322F3150E32FE91BF0E0ED5EFB
:1003B000FE4FE491A32FB0E0A559BF4FEC93391342
:1003C000F2CFE22FF0E0E659FF4F31E050916B00A1
:1003D0004081541330E0231B20938900362D353F94
:1003E000E8F5452D4330B0F480918A008F3F29F421
:1003F00080917B0080938A0006C081E0860D682E84
:10040000891708F0612C80918A008F5F8F7180932B
:100410008A0024C030917B0030938A004630C0F4BB
:1004200030918200332311F0882339F081E0860D6A
:10043000682E891798F0612C11C0862D6916D9F3A2
:10044000662019F08150682E09C02150622E06C026
:100450008111F1CF80917E00882369F3512C8FEFB9
:100460008DBD80E68CBDAA9AAA9A8FE384BB8BE1EE
:1004700087BB80EE88BB81E083BF91EA9ABD80BFD5
:100480008BB780628BBF8AB785608ABF85B7806271
:1004900085BF78948CE287B986EC86B93699FECF11
:1004A0008FEF80936000C62DC53F10F0612C3CC0DB
:1004B00080918A00803138F4E62DF0E0E559FF4F55
:1004C000C081DC2F31C05EDE80917B0080938A008A
:1004D000CDE7D0E000E010E0FF24F39481E0800F4E
:1004E0000F5F1F4F98819F3F29F421960930110516
:1004F000A9F7E2CF6DE570E097DEF801EF59FF4F05
:10050000608088818F25888377DE6FE070E080E2ED
:100510008BDE88818F258883612C6EDE33DE8091AF
:100520007D00882311F3C8CF38DE10E0F12C8CE277
:10053000D82E96ECC92EEE24EA94CE3E19F463E44C
:1005400081E204C0CD3E21F468E284E183DE76C01E
:10055000CC3E11F469E203C0CB3E19F462E581E0C0
:10056000F5CFC33F81F404E084E149DE85E090E00B
:1005700000DE88E044DE81E490E0FBDD0150A1F77D
:1005800080ED92E05AC0C43F51F584E690E0F1DD81
:10059000FCDD90E0292F30E0F901E25EFF4FE491AD
:1005A000E81710F49E5FF6CFF901E15EFF4F04916A
:1005B0006DE770E0802F82958695877035DE8EEE30
:1005C00092E0D7DD65E070E081E02EDE85E694E024
:1005D000D0DD6DE770E0802F8F7126DE0DC0CE3F3D
:1005E00071F400E00093860007DE6AEF70E081E0BE
:1005F0001BDE0F5F0A31B1F7C5DDC4DD1FC0CD3F83
:1006000069F58FEF80938700F7DD85E0F8DDBADDCF
:10061000B9DD84E1F4DD37DE80938700EDDDB2DD06
:10062000B1DDF9CF3699FECFE0926000F39490915E
:1006300087008917C8F484EF91E09BDD80917B00EF
:1006400080938A00A2DD803998F51F5F183008F486
:1006500074CFD53190F010E0DAE0CAE08D2FCFDD15
:1006600012DED7B8C6B8DECFDB3028F3F4E1FF15D1
:1006700010F7E0927B00DAE0DECFD23030F08D2F41
:1006800086958695D695D80F12C06FDD85B7877E83
:10069000806185BFF89485B7846885BF8B7F85BFEF
:1006A00085B7806285BF889585B78F7D85BFCD2F43
:1006B00010E043CF112416B858DD87B3847E87BB82
:1006C00080E061E034E0A4E040E25EE496B39A2783
:1006D000999B03C0511003C03CC0911108C025E094
:1006E000251508F038C0811136C060E039E0252DAD
:1006F00071E0273008F070E0270F522E263019F4F1
:10070000FA013197F1F7611108C0811105C081E04C
:10071000911103C080E001C081E0999895B7977E60
:10072000906195BFA895932F987011F420E401C0B3
:1007300020E6932F9770922B91BD95B7946895BF43
:100740009B7F95BF78948895F89491B59F7B91BDD8
:10075000BDCF9111CCCF8FE58DBF81E08EBF1FBE85
:10076000B1DD552011F0189501C0A4DFE199FECF4D
:100770001FBA8EBBE09A99278DB30895262FE19971
:10078000FECF1CBA1FBA8EBB2DBB0FB6F894E29AEF
:0C079000E19A0FBE01960895F894FFCF87
:00000001FF
